:1000000012C02CC02BC0FAC58EC528C027C026C080
:1000100025C024C023C022C021C020C01FC01EC0D4
:100020001DC01CC01BC011241FBECFE5D4E0DEBF25
:10003000CDBF10E0A0E6B0E0E8EDFAE102C0059027
:100040000D92AC3BB107D9F710E0ACEBB0E001C0CA
:100050001D92A53FB107E1F70CDB3CCDD1CF9298C3
:1000600093988A988B9808958A9A82E08A95F1F7F6
:1000700008958B9A82E0982F9A95F1F78A98982F95
:100080009A95F1F78B98982F9A95F1F78A9A8A9515
:10009000F1F708958B9A8A9A82E0982F9A95F1F752
:1000A0008B98982F9A95F1F78A988A95F1F7089589
:1000B00020E042E08B9A87FF02C08A9801C08A9AAA
:1000C00032E0942F9A95F1F78B98942F9A95F1F747
:1000D0002F5F283011F0880FEDCF8B9A8A98832FED
:1000E0008A95F1F78B98832F8A95F1F780B38695DF
:1000F000869580FD02C080E008958FEF0895482F17
:100100008B9A8A9882E0982F9A95F1F78B988A9526
:10011000F1F720B326952695217090E032E08B9A76
:10012000832F8A95F1F78B98832F8A95F1F7220F09
:10013000829921609F5F973091F78B9A442311F445
:100140008A9A01C08A9882E0982F9A95F1F78B9845
:100150008A95F1F7822F08950F931F93880F4130EE
:1001600071F4162F180F02E005C094DF8A9A802FD1
:100170008A95F1F7812F9CDF8F3FB9F302C0860F7C
:1001800097DF1F910F910895DC0120E040E050E0DF
:1001900098E115C0FD01E40FF51FE08138E08E2FD6
:1001A0008227F82FF17080FD29272695F13009F478
:1001B0002068315011F0E695F2CF4F5F5F4F461740
:1001C000570741F7822F0895DC01CB018115910576
:1001D000A105B10529F081509040A040B040D9F769
:1001E0000895282F30E020773070A90173E0440F84
:1001F000551F7A95E1F7220F331F420F531F94E0EA
:10020000559547959A95E1F78F70840F0895E82FDB
:10021000F0E040E050E08E2F6AE014DC292F8E2FB2
:1002200011DCE82F30E0042E02C0220F331F0A94A5
:10023000E2F7F22B4C5F5F4F4031510561F78F2F92
:1002400008950F931F93182F062F0EDF80ED30DFD8
:10025000812F2EDF802F2CDF1DDF1F910F9108953E
:10026000FF920F931F93182F062FF42EFDDE80EDC3
:100270001FDF84E01DDF812FCADF1ADF802FC7DF79
:1002800017DF8F2DC4DF14DF05DF1F910F91FF9063
:100290000895FF920F931F93F82E062F142FE4DE7C
:1002A00080ED06DF80E004DF812FB1DF01DF802FEA
:1002B000AEDFFEDE8F2DABDFFBDEECDE1F910F919C
:1002C000FF9008951F93182F137061111061411151
:1002D0001068CADE80EDECDE87E0EADE812FE8DE22
:1002E000D9DE1F9108951F93182FBEDE80EDE0DE4A
:1002F000812FDEDEB9DE81EDDBDE80E000DF182F4E
:10030000C9DE812F1F910895CF92DF92EF92FF9265
:100310000F931F938C017B016A01A6DE80EDC8DE7E
:1003200084E0C6DEB7DEA0DE81EDC2DE81E0E7DE7E
:10033000282F30E020773070A90173E0440F551F5B
:100340007A95E1F7220F331F420F531F94E0559522
:1003500047959A95E1F78F70840FF80180839ADEB4
:1003600083DE81EDA5DE81E0CADE282F30E0207734
:100370003070A90103E0440F551F0A95E1F7220FE1
:10038000331F420F531FB4E055954795BA95E1F7D7
:100390008F70840FF70180837DDE66DE81ED88DE5D
:1003A00081E0ADDE282F30E020773070A901A3E096
:1003B000440F551FAA95E1F7220F331F420F531F19
:1003C000E4E055954795EA95E1F78F70840FF601C3
:1003D000808360DE1F910F91FF90EF90DF90CF90B0
:1003E0000895CF92DF92EF92FF920F931F936C01CB
:1003F0007B018A0139DE80ED5BDE80E059DE4ADE7A
:1004000033DE81ED55DE81E07ADE282F30E0207783
:100410003070A90173E0440F551F7A95E1F7220F60
:10042000331F420F531F94E0559547959A95E1F776
:100430008F70840FF80180832DDE16DE81ED38DEAB
:1004400081E05DDE282F30E020773070A90103E0E5
:10045000440F551F0A95E1F7220F331F420F531F18
:10046000B4E055954795BA95E1F78F70840FF70181
:10047000808310DEF9DD81ED1BDE81E040DE282F78
:1004800030E020773070A901A3E0440F551FAA95F2
:10049000E1F7220F331F420F531FE4E055954795B4
:1004A000EA95E1F78F70840FF6018083F3DD1F91E9
:1004B0000F91FF90EF90DF90CF900895FF920F93F0
:1004C0001F93CF93DF93F82EFB01DA01E9018081BE
:1004D000482F50E0918180E0482B592B80E1F8169D
:1004E00071F4CA018E7F33E0880F991F3A95E1F7C6
:1004F00026814CE050E0421B5109480F591F57FF1D
:1005000006C081E08C93509541955F4F01C01C92CD
:1005100088E2F81691F48481682F70E0CB01807630
:1005200090708036910549F066FF02C04E7F05C08D
:1005300065FF02C04C7F01C0487FCA0124E0969548
:1005400087952A95E1F78883842F8F70F80180833F
:1005500080E0DF91CF911F910F91FF9008950F934D
:100560001F93DF93CF93CDB7DEB728970FB6F894DC
:10057000DEBF0FBECDBF082F162FDE011196E0E6BD
:10058000F0E088E001900D928150E1F7242F30E0F7
:1005900081E792E0BC01269FC001279F900D369F06
:1005A000900D112468EE73E06DDACB012AE0129F02
:1005B000B0011124680F791F002379F4FE013196F0
:1005C0009E01275F3F4F8081481719F46F5F7F4F6F
:1005D00004C03196E217F307B1F7CB0128960FB6A6
:1005E000F894DEBF0FBECDBFCF91DF911F910F9169
:1005F0000895882319F0709561957F4F442319F071
:10060000309521953F4F6217730714F48FEF0895CB
:1006100080E0261737070CF481E00895CF93DF932D
:10062000EC01FFD8CDD8882311F481E009C088EB14
:10063000BE01EED962E174E380E090E0C5DD80E0C8
:10064000DF91CF9108951F93CF93DF93182FEB0184
:10065000E8D8B6D8882311F482E007C084E4BE014C
:10066000D7D9113009F0B5D880E0DF91CF911F9133
:1006700008951F93CF93DF93182FEB01D2D8A0D802
:10068000882311F482E00FC088E4BE01C1D9113083
:1006900009F09FD862E174E380E090E095DD1130CD
:1006A00009F0AAD880E0DF91CF911F9108950F93B0
:1006B0001F93CF93DF93EC018B01B3D881D88823AC
:1006C00011F481E00FC08EEBBE01A2D9C0E0D0E0F2
:1006D00055D9F801EC0FFD1F80832196C930D10553
:1006E000B9F780E0DF91CF911F910F910895FF92AC
:1006F0000F931F93CF93DF93EC01162F042FF22E4D
:1007000090D85ED8882311F481E00DC08EE4BE013C
:100710007FD9812F23D9802F21D98881883211F464
:100720008F2D1CD980E0DF91CF911F910F91FF9009
:1007300008957F928F929F92AF92BF92CF92DF9255
:10074000EF92FF920F931F93DF93CF93CDB7DEB756
:1007500029970FB6F894DEBF0FBECDBF782E6B0180
:100760005A0149018EEB60E070E052D98E010F5FB3
:100770001F4F4AE0E42EF12CEC0EFD1EFFD8F801CD
:1007800081938F01EE15FF05C9F77E010894E11CE6
:10079000F11CC70169E070E0F7DC882311F083E009
:1007A00007C0872DB701A6019501840187DE80E08F
:1007B00029960FB6F894DEBF0FBECDBFCF91DF9163
:1007C0001F910F91FF90EF90DF90CF90BF90AF906F
:1007D0009F908F907F9008956F927F928F929F92BB
:1007E000AF92BF92CF92DF92EF92FF920F931F933F
:1007F000DF93CF93CDB7DEB729970FB6F894DEBF5E
:100800000FBECDBF6C015B014A0139010AD88EEBE6
:10081000B601FED88E010F5F1F4F5AE0E52EF12C76
:10082000EC0EFD1EABD8F80181938F01EE15FF058C
:10083000C9F77E010894E11CF11CC70169E070E072
:10084000A3DC882311F083E008C0F6018081B701A2
:10085000A5019401830132DE80E029960FB6F89459
:10086000DEBF0FBECDBFCF91DF911F910F91FF90E3
:10087000EF90DF90CF90BF90AF909F908F907F9040
:100880006F9008950F931F938C01CBD784EBB80121
:10089000BFD881E021D8182FC4D7111111E0812FC2
:1008A0001F910F9108950F931F93CF93DF938C01A6
:1008B000EB01F8018081BE0164D8F801808381508A
:1008C0008D3F28F48881883211F0803191F7DF91D3
:1008D000CF911F910F910895282F362F8091C1003D
:1008E0008823A1F5822F6AE0ADD88093C900822FBA
:1008F000A9D89093CA00832FA5D88093CB00832FCB
:10090000A1D89093CC00842F9DD88093CD00842FC4
:1009100099D89093CE0020E030E041E0F901E15910
:10092000FF4F9081F901E753FF4F8081F901EB52AE
:10093000FF4F891711F0408301C010822F5F3F4F96
:100940002630310559F71092C30008951092D50052
:100950001092D6001092D7001092D8001092D900B1
:100960001092DA0008950F931F93CF93DF93282FEF
:10097000362F6AE067D88093C900822F63D890939E
:10098000CA00832F5FD88093CB00832F5BD89093CE
:10099000CC00842F57D88093CD00842F53D89093C8
:1009A000CE0020E030E002E013E068EC70E0F901F6
:1009B000E753FF4F4081F901E159FF4F80818417D0
:1009C00020F4F901EB52FF4F0083F901E159FF4F89
:1009D0008081481720F4F901EB52FF4F108350E05B
:1009E000E901CB52DF4FD901A159BF4F8881823035
:1009F00031F48C91841719F08C918F5F8C938881DE
:100A0000833031F48C91841719F08C9181508C9340
:100A10008C91841751F08CEB92E0FB013197F1F748
:100A20000197D9F75F5F593009F72F5F3F4F2630A5
:100A3000310509F0BCCFDF91CF911F910F9108953F
:100A40000F931F93CF93DF93EC0125E030E06AE032
:100A500048EC50E08091700080936F0080917100AD
:100A60008093700080917200809371008091730078
:100A7000809372008091740080937300F901E159B2
:100A8000FF4F608388EE93E0FA013197F1F7019709
:100A9000D9F7215030402223E9F68AE080936F0095
:100AA000CE0164E670E0DAD7062FCE016AE070E08E
:100AB000D5D7CB016AE070E0D1D7182FCE016AE01C
:100AC00070E0CCD725E030E09AE068EC70E0F90106
:100AD000E159FF4F0083F901E059FF4F1083F901FD
:100AE000EF58FF4F8083F901EE58FF4F908348EE97
:100AF00053E0FB013197F1F741505040D1F72150BD
:100B000030402130310519F78091AF00813031F448
:100B100080917B008093680010926F00DF91CF91ED
:100B20001F910F9108951F920F920FB60F921124EB
:100B30002F933F934F935F938F939F93AF93BF9365
:100B4000CF93DF93EF93FF9315BAC69AE091C40059
:100B5000F0E0E859FF4F808183BD4091C3004931E7
:100B6000E0F58091C5008F5F8093C5008231A9F5C3
:100B70001092C50050917A0020E030E0842F90E080
:100B8000EC01CB56DF4FDC01A458BF4FF901EB520B
:100B9000FF4F8081813011F0442349F4F901E85975
:100BA000FF4F513011F48C9101C0888180834C300B
:100BB00061F48091C100882341F4F901E753FF4FAC
:100BC0008081F901E159FF4F80832F5F3F4F26302D
:100BD0003105E1F64F5F4093C300FF91EF91DF9144
:100BE000CF91BF91AF919F918F915F914F913F9125
:100BF0002F910F900FBE0F901F9018951F920F927C
:100C00000FB60F9211245F936F937F938F939F93EF
:100C1000AF93BF93EF93FF939091C4009630E0F5AC
:100C2000E92FF0E0DF01A159BF4F8C91833061F0D3
:100C30008C91843049F08C91873031F08C918930DF
:100C400019F08C918A3011F4C09A01C0C098E15912
:100C5000FF4FE081F0E0E055FF4F808182BB923092
:100C600091F0933028F4992351F09130E1F409C0C8
:100C7000943069F0943048F09530A9F40AC080E2CD
:100C800009C080E107C088E005C084E003C081E0BE
:100C900001C082E085BB07C0963029F480917900BD
:100CA000813009F4C698892F8F5F8093C400873004
:100CB00010F01092C4008091C200882369F0849BD8
:100CC00002C08AE007C08091C6009091C7006AE028
:100CD00070E0C4D680937300FF91EF91BF91AF9104
:100CE0009F918F917F916F915F910F900FBE0F90A9
:100CF0001F9018958091BF00882319F18091C10041
:100D00008330F8F42091D300822F6AE09BD6809341
:100D10006F00822F97D6909370002091DC00822F75
:100D200091D680937100822F8DD69093720020917E
:100D3000D200822F87D680937300822F83D6909320
:100D400074008091BF00882319F18091C100833025
:100D5000F8F02091DB00822F6AE074D680936F0058
:100D6000822F70D6909370002091ED00822F6AD66A
:100D700080937100822F66D6909372002091D400E8
:100D8000822F60D680937300822F5CD6909374007C
:100D90008091C100833009F477C0843030F4813011
:100DA00059F0823009F02BC13BC0843009F4AEC049
:100DB000853009F024C1ECC0B49912C08091D300F1
:100DC0008F5F8093D300883110F01092D3008CEDA8
:100DD00095E028EC30E0F9013197F1F70197D9F768
:100DE000B59915C08091D30081508093D300B599F7
:100DF00005C0882319F487E18093D3008CED95E03A
:100E000028EC30E0F9013197F1F70197D9F784998F
:100E100004C0B59B02C0B49973C02091D30066C0D2
:100E2000B49912C08091DC008F5F8093DC008C331A
:100E300010F01092DC008CED95E028EC30E0F90128
:100E40003197F1F70197D9F7B59915C08091DC007A
:100E500081508093DC00B59905C0882319F48BE399
:100E60008093DC008CED95E028EC30E0F9013197BF
:100E7000F1F70197D9F7849904C0B59B02C0B499E2
:100E800081C02091DC0074C0B49913C08091DB0054
:100E90008F5F8093DB00803218F081E08093DB006D
:100EA0008CED95E028EC30E0F9013197F1F70197EE
:100EB000D9F7B59913C08091DB0081508093DB0096
:100EC000882319F48FE18093DB008CED95E028EC0A
:100ED00030E0F9013197F1F70197D9F7849904C00F
:100EE000B59B02C0B4990CC02091DB00822F6AE050
:100EF000A9D580936F00822FA5D590937000089597
:100F00008AE080936F00809370000895B49913C0B5
:100F10008091ED008F5F8093ED008D3018F081E0BF
:100F20008093ED008CED95E028EC30E0F9013197ED
:100F3000F1F70197D9F7B59913C08091ED00815071
:100F40008093ED00882319F48CE08093ED008CED04
:100F500095E028EC30E0F9013197F1F70197D9F7E6
:100F6000849904C0B59B02C0B4990CC02091ED00D7
:100F7000822F6AE067D580937100822F63D59093AA
:100F8000720008958AE08093710080937200089542
:100F9000B4990EC08091D4008F5F8093D4008CED03
:100FA00095E028EC30E0F9013197F1F70197D9F796
:100FB000B5990EC08091D40081508093D4008CEDFF
:100FC00095E028EC30E0F9013197F1F70197D9F776
:100FD000849904C0B59B02C0B4990CC02091D40080
:100FE000822F6AE02FD580937300822F2BD59093A8
:100FF000740008958AE080937300809374000895CC
:101000008BED90E06DEE70E044ED50E07DD9809185
:101010007B00809368008093690080936A008093CE
:101020006B0080936C0080936D008091DB00609179
:10103000ED004091D40097DC089583ED90E06CEDD5
:1010400070E042ED50E0CDD98091D3006091DC009A
:101050004091D20041DC089580916F00882351F5C2
:1010600020E030E06AE048EC50E08091730080932B
:10107000740080917200809373008091710080935E
:101080007200809170008093710080916F00809356
:101090007000F901E159FF4F608388EE93E0FA0197
:1010A0003197F1F70197D9F72F5F3F4F2630310580
:1010B000E1F625C020E030E06AE048EC50E08091A5
:1010C000730080937400809172008093730080910C
:1010D0007100809372008091700080937100F9011B
:1010E000E159FF4F608388EE93E0FA013197F1F701
:1010F0000197D9F72F5F3F4F2430310501F783ED7A
:1011000090E06CED70E042ED50E06BD92091D3009F
:10111000822F6AE097D48093C900822F93D4909352
:10112000CA002091DC00822F8DD48093CB00822FC7
:1011300089D49093CC002091D200822F83D48093C5
:10114000CD00822F7FD49093CE00AEECB0E028EC9F
:1011500030E08091730080937400809172008093DE
:101160007300809171008093720080917000809371
:10117000710080916F00809370008C9180936F005C
:1011800088EE93E0F9013197F1F70197D9F71197BC
:1011900080E0A83CB807E9F608950F931F938C01EF
:1011A00080917B00809368008093690080936A003F
:1011B00080936B0080936C0080936D0081E060E011
:1011C00070E041DA03521F4FF80180818093CF0015
:1011D0006FEA70E04EEA50E021ED30E0AADA8823B1
:1011E00031F08FEF8093AE0081E08093AF0080916B
:1011F000AF006091AE004091D100B1D99093C7008B
:101200008093C6001DDC81E08093C2001F910F9186
:101210000895B49938C08091C100882329F4809141
:10122000C0008F5F8093C0008091C0008A3009F5B4
:1012300080917900813061F41092790088EE93E01A
:1012400028EC30E0F9013197F1F70197D9F70CC09C
:1012500081E08093790088EE93E028EC30E0F9019A
:101260003197F1F70197D9F76091790080E090E02C
:1012700024D488EE93E028EC30E0F9013197F1F7BF
:101280000197D9F71BC08091C0008823A9F08091F5
:10129000C0008A3088F48AE08093C100B1DE80E229
:1012A0009EE428EC30E0F9013197F1F70197D9F786
:1012B0001092C1001092C0001092C000B5992BC0CE
:1012C0008091C100882339F58AE08093C100809124
:1012D000D000882319F080E090E05FDF80E29EE498
:1012E00028EC30E0F9013197F1F70197D9F78091B7
:1012F000D000823061F481E090E04FDF80E29EE434
:1013000028EC30E0F9013197F1F70197D9F7109205
:10131000C1001092C200B3995CC08091BF008F5F82
:101320008093BF008091C100823031F48091D3005E
:101330006091DC0040E0ADD78091BF00813049F47E
:101340008091C100882329F08091C1008F5F809334
:10135000C1008091BF008A30A9F48091C100882328
:1013600089F481E08093C1001092790080ED97E0CC
:1013700028EC30E0F9013197F1F70197D9F781E0D6
:10138000809379008091C1008630C8F01092790076
:1013900088EE93E028EC30E0F9013197F1F70197FE
:1013A000D9F781E0809379008091DB006091ED00B6
:1013B0004091D40055D71092C1001092BF0088EE22
:1013C00093E028EC30E0F9013197F1F70197D9F774
:1013D00008958091C100882399F58091BF008823EA
:1013E00079F1809178008F5F809378001092BE0031
:1013F00080917800843010F0109278009AE09093F9
:10140000C10090936F0090937000109271008091D2
:1014100078008F5F809372009093730090937400B4
:1014200088E893E128EC30E0F9013197F1F7019772
:10143000D9F71092C1006091780081E090E03DD32F
:101440001092BF00089580917800813051F0813072
:1014500030F0823021F1833009F0ABC059C0EDDDAE
:1014600054C08091BE00893708F4E7DD8091BE004A
:10147000893709F4C5DD8091BE00833808F499C02E
:1014800083ED90E06CED70E042ED50E0AAD78091E2
:10149000D3006091DC004091D20065DA36C08091C3
:1014A000BE00893708F4C9DD8091D000882381F01F
:1014B000813081F48091BE00893719F480E090E09A
:1014C0006CDE8091BE00833828F01092C200C4DD2B
:1014D0001092BE008091D000823009F06AC08091E5
:1014E000BE00893719F480E090E057DE8091BE009D
:1014F000833819F481E090E050DE8091BE008D3891
:1015000008F457C01092C200A7DD1092BE000895E3
:101510008091BE00893708F490DD8091BE00893744
:1015200009F46EDD8091D0008823A1F48091BE0083
:10153000833880F083ED90E06CED70E042ED50E098
:1015400050D78091D3006091DC004091D2000BDA3B
:101550001092BE008091D000813081F48091BE0055
:10156000833819F480E090E018DE8091BE008D3859
:1015700028F01092C20070DD1092BE008091D00061
:101580008230B9F48091BE00833819F480E090E095
:1015900004DE8091BE008D3819F481E090E0FDDD1D
:1015A0008091BE00873928F01092C20055DD10925C
:1015B000BE0008958F929F92AF92BF92DF92EF92FA
:1015C000FF920F931F93DF93CF93CDB7DEB7299789
:1015D0000FB6F894DEBF0FBECDBF8FEF898300E05A
:1015E00010E022E0E22EF12CEC0EFD1E4E010894DC
:1015F000811C911C9AE0A92EB12CAC0EBD1E1FC0FF
:10160000C401B70150D989818F3F19F08E3F39F459
:101610008FEF8093AE0081E08093AF0017C0D701B9
:10162000F80183E0EE0FFF1F8A95E1F7E352FF4FC9
:101630008D918193AA15BB05D9F70F5F1F4FD02E4F
:101640008981882319F002301105D1F68D2D299654
:101650000FB6F894DEBF0FBECDBFCF91DF911F91C3
:101660000F91FF90EF90DF90BF90AF909F908F9081
:101670000895EF92FF920F931F9384B38F6384BBFF
:1016800087B3816487BB81B3806E81BB85B583607E
:1016900085BD89B7806C89BFE2D480E061E041E01C
:1016A00011D686E390E068E370E047E350E021E084
:1016B000FCD080DF8093D000882321F081E060E0BF
:1016C00070E0C1D788EE93E028EC30E0F901319763
:1016D000F1F70197D9F782E090E0E7D1813061F02E
:1016E00080E090E061E0E9D181E090E063E0E5D165
:1016F00082E090E061E0E1D180E090E0D6D180939B
:10170000790081E090E0D1D18093780078949AE0DC
:101710009093C10090936F009093700010927100AD
:10172000809178008F5F8093720090937300909304
:10173000740080E29EE428EC30E0F9013197F1F783
:101740000197D9F71092C1008BED90E06DEE70E03B
:1017500044ED50E0D9D5EE24E3941AE039E6F32EB7
:1017600008EC8091C1008111C5DA53DD849B25C04E
:101770008091C100882309F58091BC00882389F7F6
:101780008091BC008F5F8093BC008091BE008F5F12
:101790008093BE008091D300873038F410927A0095
:1017A000F0927B0000936E0006C0E0927A001093E6
:1017B0007B0010936E0047DED4CF1092BC00D1CFD7
:1017C000E091F100F091F20080819091F000892386
:1017D0000895E091EE00F091EF0080819091F0008B
:1017E000892B8083E091F300F091F4008081909147
:1017F000F000892B80830895E091EE00F091EF00D6
:1018000090818091F000809589238083E091F3009E
:10181000F091F40090818091F0008095892380837D
:101820000895E091EE00F091EF0090818091F0003A
:10183000809589238083E091F300F091F40080810A
:101840009091F000892B80838FEB93E081159105B7
:1018500011F00197F1F72FB7F894E091F300F091B0
:10186000F40090818091F00080958923808383E843
:1018700090E08115910511F00197F1F7E091F100E9
:10188000F091F20040813091F0002FBF8BE393E0A4
:101890008115910511F00197F1F78081832311F4EF
:1018A00081E00895842F832308955093F40040939A
:1018B000F3007093EF006093EE009093F20080933A
:1018C000F10081E090E002C0880F991F2A95E2F7AD
:1018D0008093F000A6DF0895382F4FB7F894E09179
:1018E000F300F091F40080819091F000892B8083C7
:1018F00081E090E08115910511F00197F1F7332314
:1019000051F0E091F300F091F40090818091F000AB
:1019100080958923808389E190E08115910511F0FC
:101920000197F1F7E091F100F091F20080812091B0
:10193000F000822309F430E089E590E081159105FB
:1019400011F00197F1F7E091F300F091F40080813C
:101950002095282320834FBF832F08950F931F9333
:10196000182F08E0812F8170B7DF1695811110685C
:101970000150C1F7812F1F910F9108958FEFEEDF76
:101980000895DF92EF92FF920F931F93CF93DF930F
:10199000E82EEB0146DF882381F580EFDFDF80E46E
:1019A000FF24182F98EFD92ED80E81E095DF082F4D
:1019B00081E092DF882329F0002371F08EEFF82E6A
:1019C0001EC0002349F41E1528F0888180FF04C042
:1019D000E11611F0F12E01E0802F7EDF88818695DF
:1019E0008883002311F08068888311501D15E9F663
:1019F000112329F02196812FD4CFFF24FA948F2D23
:101A0000DF91CF911F910F91FF90EF90DF9008959C
:101A10000F931F93CF93DF93082FEB0102DF2097E3
:101A200041F085E59BDF18E0899198DF1150E1F7DF
:101A300002C08CEC93DF802F91DFDF91CF911F915B
:101A40000F910895991B79E004C0991F961708F02B
:101A5000961B881F7A95C9F780950895AA1BBB1B12
:101A600051E107C0AA1FBB1FA617B70710F0A61B9E
:101A7000B70B881F991F5A95A9F780959095BC01BF
:101A8000CD01089597FB092E07260AD077FD04D0D3
:101A9000E5DF06D000201AF4709561957F4F089518
:101AA000F6F7909581959F4F0895E199FECF9FBBE2
:101AB0008EBBE09A99278DB30895262FE199FECF2A
:101AC0009FBB8EBB2DBB0FB6F894E29AE19A0FBE76
:081AD00001960895F894FFCF80
:101AD80001030406090B0C0E010101010101010AB1
:101AE8000A0A0A0A0A000000020101FA01152A3F3F
:101AF80054697E93A8BDD2E7F5E7D2BDA8937E6965
:101B0800543F2A150169747F8A95A2AFBAC6D2DEFE
:101B1800EAF5EADED2C6BAAFA2958A7F7469FF01F8
:0C1B2800604080A000200020A080E000B1
:00000001FF
